:020000040000FA
:06000000A0EF23F0120046
:020006001200E6
:0600080004EF08F01200F5
:02000E000014DC
:07001000032A2C010100008E
:060018000CEF08F01200DD
:02001E000200DE
:10002000BB470000910500005D0000000E000000CD
:08003000EE05000009000000CC
:0800380058EC05F0FB0EDBCFD4
:10004000F3FFDB06F35000090AE0A6EC05F0FA0E18
:1000500011EC06F0F3E1261CF1E1010E01D0000ED7
:1000600087EF05F058EC05F03B0EE12402E3E16870
:10007000E652E16E010EDB6A020EDB6AF90EDBCF9F
:10008000F6FFFA0EDBCFF7FFFB0EDBCFF8FF080021
:10009000F550DF6EDF5002E1ABEF04F0250EDF5CC0
:1000A00002E09EEF04F0030EDB6A040EDB6A050E2D
:1000B000DB6A060EDB6A070EDB6AC0EC04F02D0E6D
:1000C000DF5C0CE02B0EDF5C09E0200EDF5C06E05D
:1000D000230EDF5C03E0300EDF5C1AE1DF50300AF4
:1000E00014E0130A0FE0030A0AE00B0A05E0060A0F
:1000F000E4E1030EDB80E1D7030EDB82DED7030EE3
:10010000DB84DBD7030EDB86D8D7030EDB88D5D79D
:100110002A0EDF5C1BE1BCEC04F00AEC05F010E0F9
:10012000030EDB8006680768130EDBCF0DF0140E9C
:10013000DBCF0EF039EC23F0040E04C0DBFF03D05C
:10014000130EF3EC04F0C0EC04F00BD0090EDB6AE4
:1001500061EC05F003E0D5EC05F0FAD7090EF3ECFD
:1001600004F0030EDBB0DB982E0EDF5C1BE1C0EC6D
:1001700004F02A0EDF5C0BE1BCEC04F00AEC05F0A5
:1001800003E1130E45EC05F0C0EC04F00BD0090EB2
:10019000DB6A61EC05F003E0D5EC05F0FAD7090E57
:1001A00045EC05F0680EDF5C07E1C0EC04F0680E7A
:1001B000DF5C1DE1030E18D0740EDF5C17E07A0ED1
:1001C000DF5C14E0480EDF5C06E0540EDF5C03E009
:1001D0005A0EDF5C02E1020E07D06C0EDF5C03E01A
:1001E0006A0EDF5C04E1010E98EC05F0C9DBDF501C
:1001F0006E0A01E17FD31E0A01E192D1200A01E1DA
:100200008FD13F0A01E149D11A0A01E146D10D0A15
:1002100001E143D1200A01E140D13A0A01E13DD197
:10022000200A01E13AD1260A01E135D10D0A01E1A6
:1002300032D11A0A01E1D9D0200A4AE0300A1FE07F
:10024000460A0EE0250A01E083D3D950F90FE96E82
:10025000FF0EDA20EA6E010EEE5E000EEE5AEE5A46
:10026000A6EC05F0250EE66E95DB03E1261C01E108
:1002700069D3A2EC05F001E26BD3DB2A69D3080E47
:10028000DB6A040EDB50010806E2040EDB046AECB4
:1002900005F0DB508BDB080EDB5009E0030EDB5072
:1002A000010B05E172DB01E04DD3080EDB6A64DB74
:1002B000EFCFDFFF1AEC06F003E1261C01E142D389
:1002C000A2EC05F001E3DB2A60DB01E141D33AD384
:1002D000070EDB5002080FE1E6EC05F0030EADEC73
:1002E00005F00E0EEECFDBFF0F0EEECFDBFF100E94
:1002F000EECFDBFF20D0F70EDBCF28F0F80EDBCF00
:1003000029F0020E285E000E295AF70E28C0DBFFE6
:10031000F80E29C0DBFF28C0E9FF29C0EAFF9DECE9
:1003200005F0276A0E0E25C0DBFF0F0E26C0DBFF8F
:10033000100E27C0DBFF0E0EDBCFE6FF0F0EDBCF6C
:10034000E6FF100EDBCFE6FFFAEC20F0E552E552B7
:10035000E552130E05C0DBFF140E06C0DBFF060ED0
:10036000DB5005E0130EE1EC05F001E26ADB05EC81
:1003700006F002E2130E37DBC8EC05F006E0040ECF
:10038000E1EC05F002E2050E2EDB030EDBB005D03A
:10039000FCDA01E0D7D2080EDB6A090EDB6A0E0E2A
:1003A000DBCFF6FF0F0EDBCFF7FF100EDBCFF8FF32
:1003B0000800F550DF6EDF5014E00BEC06F011E2A0
:1003C0001AEC06F003E1261C01E1BCD2BBDB01E321
:1003D000DB2A090EDB2AD9500E0FE96E000ECBDBAB
:1003E000E7D7D3DA01E1B4D2ADD2C6DA110EEECF3F
:1003F000DBFF120EEDCFDBFF110EDBCFE6FF120E9F
:10040000DBCFE6FF40EC21F0E552E552130EF3CFCF
:10041000DBFF140EF4CFDBFF060EDB5004E0130EFF
:10042000D0DB01E20EDB05EC06F002E2130EDBDAB4
:10043000AFDB05E0040EC5DB02E2050ED4DA030EE5
:10044000DBB005D0A2DA01E07DD2080EDB6A090E2E
:10045000DB6A110EDBCFE9FF120EDBCFEAFFEFCF35
:10046000DFFFDF5014E0D7DB12E2E4DB03E1261C00
:1004700001E168D267DB01E3DB2A090EDB2A110EFA
:10048000DB2ADBCFE9FF120EE8E3DB2AE6D77DDAD1
:1004900001E15ED257D2030EDB8E070EDB0410E1C2
:1004A00095DB040E5ADB0A0EEECFDBFF0B0EEECF10
:1004B000DBFF0C0EEECFDBFF0D0EEECFDBFF6CD0C3
:1004C000070EDB5003082CE1030EDBAE0DD0B2DAD1
:1004D000020E76DAEFCF25F0266A276A286A25AE63
:1004E00039D02668276835D0F70EDBCF26F0F80E16
:1004F000DBCF27F0020E265E000E275AF70E26C02D
:10050000DBFFF80E27C0DBFF26C0E9FF27C0EAFFAC
:10051000EFCF25F00A0E25C0DBFF0B0EDB6A38D0CB
:10052000070EDB50020809E1030EDBAE04D059DBF5
:1005300027AE10D00ED055DB0DD0030EDBAE12D09F
:1005400079DA020E3DDAF9DA276A286A26AE02D095
:1005500027682868E2DA0C0E27C0DBFF0D0E28C0E2
:10056000DBFF1AD0F70EDBCF27F0F80EDBCF28F039
:10057000020E275E000E285AF70E27C0DBFFF80E8A
:1005800028C0DBFF27C0E9FF28C0EAFFD6DAC5DABA
:100590000C0EDB6A0D0EDB6A060EDB5005E1010E68
:1005A000F36E050EF3CFDBFF150EDB6A160EDB6A6A
:1005B000D950370F256E000EDA20266E390E25C071
:1005C000DBFF3A0E26C0DBFF380EDB6A080EDB6A63
:1005D0000A0EAEDADF50780A12E0200A10E0280A8C
:1005E0000CE0200A0AE03F0A06E00D0A02E0200AB9
:1005F00008E1020E05D0080E03D0080EDF26100E0B
:1006000097DA030EDBBE02D0DB92DB94DB50800B6B
:1006100024E08ADAD890030EEB50000A08E6000EB8
:10062000EE5C000EEE58000EEE58000EEE5815E28D
:1006300013DA0B680C680D680E6801EC23F00A0EE3
:1006400000C0DBFF0B0E01C0DBFF0C0E02C0DBFFA6
:100650000D0E03C0DBFF2D0E08D0030EDBA202D06F
:100660002B0E03D0DBA408D0200EF36E170EF3CFB1
:10067000DBFF150EDB2A02D0170EDB6A050EDB50FE
:1006800003E1B7D901E189D0AA0E256E470E266E87
:10069000000E276E070EDBCF28F0296A2A6A2B6A24
:1006A00028C00BF029C00CF02AC00DF02BC00EF0B2
:1006B000D3D9DBEC07F025500024F36E265001203F
:1006C000F46E27500220F86EF4CFF7FFF3CFF6FF59
:1006D0000800090EF5CFDBFF580EDF5C0FE1610E5D
:1006E000F36E090E7BD90AE3200E256E090EDBCFCF
:1006F000E7FF2550E75E090EE7CFDBFF070EDBCFF4
:1007000025F0266A276A286A0FDA25C00BF026C072
:100710000CF027C00DF028C00EF0EECF04F0EECFA5
:1007200005F0EECF06F0EFCF07F0DBEC07F007C0E7
:10073000EDFF06C0EDFF05C0EDFF04C0EFFF390E71
:10074000DBCFE9FFDB063A0EDBCFEAFF01E2DB0697
:10075000090EDBCFEFFF150EDB2A4BD995E1030E17
:10076000DBA61DD06F0EDF5C06E1C1D918E3150EC4
:10077000DB285BDA14D0780EDF5C09E0580EDF5C12
:1007800006E0620EDF5C03E0420EDF5C08E1020E71
:10079000F36E160EF3CFDBFF02D0150EDB6A030EED
:1007A000DB50100B0EE0040EDBCF25F0050EDB5006
:1007B000D880255406E2060EDB5003E1040EDB5020
:1007C00034DA95D90AE2050EDBCFE7FF150EDB50D0
:1007D000E75E050EE7CFDBFF02D0050EDB6A040EF5
:1007E000DBCF25F0160E45D9D880255414E2160E1D
:1007F000DBCFE6FF150EDBCFE6FF040EDBCFE6FF17
:10080000050EDB50E552E75CE552D880E754E5522F
:10081000D880E7545FD9030EDB50010B0BE1080EC3
:10082000DB5008E0B2D801E08DD0080EDB50BED816
:10083000080EDB6A170EDB5007E088D9170EF1D9D6
:1008400003E1261C01E17ED0160EDB5016E07ED9B6
:10085000300EE66E9FD802E1261C74E077D9DFCF18
:10086000E6FFBFEC22F0E552E552E552F4CF26F068
:100870000001F31C02E1261C65E0050EDBCF25F02C
:10088000160EDB50D880255409E2050EDBCFE7FFBA
:10089000160EDB50E75E050EE7CFDBFF300EE66E8F
:1008A000050ECBD94FE1390EDB2ADBCFE9FF3A0E3B
:1008B00001E3DB2ADBCFEAFF090EEFCFDBFFDB50E2
:1008C0000EE044D9090EADD902E1261C3BE0390EF9
:1008D000DB2ADBCFE9FF3A0EEDE3DB2AEBD755D875
:1008E00031E1160EDBCFE6FF080EC3D8E552E72450
:1008F0005DD82ED0070EDB50030A1CE0010A14E07D
:10090000030A07E07BD9DBCFEEFF020EDBCFEDFF62
:100910001FD0F5D82A6A28AE02D029682A682CD8B8
:10092000BCD82AC0EEFF14D0EAD828BE296824D843
:10093000B4D80ED063D9DBCFEFFF0AD07BD905E165
:10094000261C03E1F368F46810D0FCD801E3DB2A2D
:1009500079D947EF00F0010EDBCF25F0020EDBCF97
:1009600026F025C0F3FF26C0F4FF3B0EE15C02E257
:10097000E16AE552E16ECBD029D9020EADEF05F068
:1009800061D90800F550DF6E1200200EE66E080EE9
:100990001DEF06F0BFEC22F0E552E552E552F3CF31
:1009A00025F0F4CF26F00001F31C1200256E266A14
:1009B000D950010F4DD92550EE262650ED221200B8
:1009C000295E000E2A5AF70E29C0DBFFF80E2AC056
:1009D000DBFF29C0E9FF2AC0EAFF1200DBCFF4FFEA
:1009E000F350F45C1200DB50E76E040EE7CFDBFF40
:1009F00012000A0EDBCF25F00B0EDBCF26F00C0E1B
:100A0000DBCF27F00D0EDBCF28F025502610271066
:100A100028101200130EEECFDBFF140EEDCFDBFF1C
:100A2000130EDBCF25F0140EDBCF26F00001800E75
:100A300026141200F70EDBCF29F0F80EDBCF2AF0D8
:100A40001200050EDB50E66ED950130F01D9E552A6
:100A5000E750EE6EED6A12000A0EDBCF04F00B0ECB
:100A6000DBCF05F00C0EDBCF06F00D0EDBCF07F071
:100A70001200DBCFE6FF150EDBCFE6FF050EDB50E5
:100A8000E552E724E552E7241200DB50CED8010EF0
:100A9000F36E060EF3CFDBFF1200EE50EFCFEAFF4E
:100AA000E96E27C0EEFF28C0EEFF29C0EEFF12005E
:100AB000D9CFE6FFDACFE6FFE1CFD9FFE2CFDAFF09
:100AC0001200DFCFE6FFE66A7EEC23F0E552E55246
:100AD000F3501200E76E080EE7CFDBFF1200EECFF7
:100AE00025F0EECF26F0EFCF27F0286A1200050E92
:100AF000DBCF25F0150EDB50D88025541200010EF7
:100B0000DBCF27F0020EDBCF28F0296A1200E55276
:100B1000E5CFDAFFE7CFD9FF12000A0E25C0DBFFD1
:100B20000B0E26C0DBFF1200D9500A0F28EF06F08B
:100B3000F36E070EF3CFDBFF1200EECF25F0EFCF01
:100B400026F01200010EDB2A020E1200FC0EDBCF93
:100B5000E6FFFD0EDBCFE6FF1200255E000E265AF3
:100B6000F70E25C0DBFFF80E26C0DBFF25C0E9FF2E
:100B700026C0EAFF1200DA20EA6EEF2AEECFF6FF77
:100B8000000EEF22EECFF7FFEF22EECFF8FF1200BC
:100B9000040EDBCFE6FF130EDB50E552E75C9ADF75
:100BA000DB5004DF060EDB501200090EDB500A0D8D
:100BB000F350DF24D00FE76E090EE7CFDBFFC0EF65
:100BC00004F0DB50F36E050EEEEF04F0F70EDBCF12
:100BD00025F0F80EDBCF26F01200DFCFE6FFCAEFDC
:100BE00004F028DF030EECDE6FEF05F01CEC00F0E4
:100BF000E552E552E552E55200091200BDDEEE5025
:100C0000EFCFEAFFE96E010E1200130EDB50F36E18
:100C1000040EEEEF04F0040EDB50F36E090EEEEF5F
:100C200004F0DBCFE6FFCAEF04F0E76E050EE7CF76
:100C3000DBFF12008BDFEDEF05F0DBCFE6FF86DF99
:100C4000F6EF05F0D950F90FE96EFF0EBBEF05F096
:0A0C5000E96E000EDA20EA6E1200D1
:060C5A00DACFE4FFE652D0
:100C6000E552E5CFDAFF1100D8CFE4FFE0CFE4FF93
:100C7000E46EDACFE4FFE652E552E5CFDAFFE55065
:100C8000E5CFE0FFE5CFD8FF10003FD84EEC21F0D4
:100C90000101E26BE36B010EE46FDA0EE66E3F0ECC
:100CA000E66EE70E256E3F0E266E276A25C0E6FF2C
:100CB000E66E27C0E6FF000EE66E010EE66E1AEC49
:100CC00022F0286E070EE15E2850000EE66E010E3F
:100CD000E66E95EC21F0E552E552400EE66EE66ACE
:100CE000E66A800EE66E010EE66EE0EC20F0256E00
:100CF000050EE15E25500101800EC06F010EC16F2F
:100D0000B1EC12F057EC07F0FBD70F0EC11206D86A
:100D100025EC12F0080E146EB1EF1DF00101EC6B22
:100D2000EB6B010EEA6F12000501F551F61104E1BB
:100D3000100EF56F270EF66FF507000EF65B6DA22D
:100D400007D0F551F6112EE18B7C8BBC13D027D048
:100D50000201725102E18B9C22D0720502E18B8C60
:100D600009D0020E725D02E18B8C19D0040E725D07
:100D700003E18B9C8B8E1200100E725D06E1050163
:100D8000F551F6110FE18B7C0AD0200E725D0AE15D
:100D90000501F551F61106E18B7C8BAC02D08B9EE0
:100DA00012008B8E1200120012000101EB5109E1BA
:100DB000EC5102E0EC071200010EEB6F640EEC6FD9
:100DC0001200EC5101E0EC07120012004DEF1BF095
:100DD00012009BEF1BF0020196051EE10201970530
:100DE0001BE1E2DF6D920201976B0101100EED6FC6
:100DF0000E0EEE6FED07000EEE5BED51EE11FAE117
:100E00006D84080EED6F070EEE6FED07000EEE5BC2
:100E1000ED51EE11FAE16D941200D9CFE6FFE1CF6A
:100E2000D9FFFD0EDBCF06F0FE0EDBCF07F0050E7F
:100E3000061801E1075036E0E868061802E17F0E67
:100E400007182FE0030E061801E1075028E0020EF4
:100E5000061801E1075021E0010E061801E10750D4
:100E60001AE0740E061801E1075013E0750E06181B
:100E700001E107500CE0730E061801E1075005E090
:100E8000720E06180FE107500DD08FDF0BD08BDFED
:100E900009D08ADF07D09DDF05D09ADF03D096DF27
:0E0EA00001D093DF010EE552E7CFD9FF12001B
:020EAE00D9CF9A
:100EB000E6FFE1CFD9FF060EE126200E0201E76E24
:100EC0007219E8AE02D0E73402D0E750725D69E3F0
:100ED0006D50020B66E10001E35142E1400EE66E07
:100EE000E66AE66A400EE66E010EE66EE0EC20F081
:100EF000256E050EE15E2550400EE66E400EE66E54
:100F0000010EE66E14EC1CF0E552E552E552DE6E81
:100F1000DD6AD9CFE9FFDACFEAFFEE50ED1020E02D
:100F2000000EE66E020EE66EDECFE6FFDDCFE6FFD8
:100F3000800EE66E010EE66EDECFE6FFDDCFE6FF49
:100F4000400EE66E010EE66E0FEC08F0256E0A0EFE
:100F5000E15E2550020EF3CFDBFF030EF4CFDBFF83
:100F60000CEC1DF00CEC1DF00001E35118E1010E3A
:100F7000185C15E2176AB6EC1EF0175000080FE275
:100F80000001E3510CE11750E66E400EE66E040ED0
:100F9000E66E74EC1CF0E552E552E552176A0CEC73
:100FA0001DF0060EE15C02E2E16AE552E16EE552F7
:060FB000E7CFD9FF12009B
:0A0FB600036A026A016A006A200E55
:100FC000E76ED89004360536063607360036013609
:100FD000023603360B50005C0C5001580D5002587D
:100FE0000E50035809E30B50005E0C50015A0D508F
:0E0FF000025A0E50035A042AE72EE4D71200CC
:020FFE001200DF
:06100000A0EF23F0120036
:02100600FFFFEA
:061008002DEF06F01200BE
:021016000001D7
:0610180034EF06F01200A7
:02101E00D9CF28
:10102000E6FFE1CFD9FF0D0EE126FD0EDBCF06F086
:10103000FE0EDBCF07F0090E06C0DBFF0A0E07C06D
:10104000DBFF070EDB6A080EDB6A050EDB6A060EA5
:10105000DB6A050EDBCF25F0060EDBCF26F0FB0E9C
:10106000DBCF27F0FC0EDBCF28F02750255C285083
:10107000265801E36AD2090EDBCFE9FFDB2A0A0E0C
:10108000DBCFEAFF01E3DB2AEFCFDFFF0501EE5103
:10109000030A01E1E8D1010A01E1CAD1030A01E131
:1010A000BBD1010A01E03FD21B0EDF5C02E1010E61
:1010B00004D02B0EDF5C03E1020EEE6F3FD20D0E6B
:1010C000DF5C04E00A0EDF5C01E0FBD0F90EDBCF51
:1010D00025F0FA0EDBCF26F00101C051255CC1518D
:1010E000265801E32BD214A61FD00401320EC06F84
:1010F000050EC16F3F0EC26F550EC36F200E050166
:10110000EF250401C46FC56BDDEC1DF00A0EE66E21
:10111000CAEC23F0E5520CEC1DF0010EE66EDDEC9E
:101120001FF0E552DDEC1DF0030EDB6A040EDB6AF6
:10113000F90EDBCF06F0FA0EDBCF07F00B0E06C080
:10114000DBFF0C0E07C0DBFF400EE66EE66AE66AC8
:10115000C00EE66E040EE66EE0EC20F0256E050E85
:10116000E15E25500401200EC06F0B0EDBCF25F091
:101170000C0EDBCF26F00101C051255CC151265871
:1011800026E20B0EDBCFE9FF0C0EDBCFEAFFEF50C0
:10119000E66E020EE76E030EDBCFE9FF040EDBCF37
:1011A000EAFFE750E926000EEA22C00EE926040E07
:1011B000EA22E552E750EF6E0B0EDB2A0C0E01E33C
:1011C000DB2A030EDB2A040ED0E3DB2ACED705018F
:1011D000F05102E0F00517E1020EE76E030EDBCFDF
:1011E000E9FF040EDBCFEAFFE750E926000EEA2212
:1011F000C00EE926040EEA220D0EEF6E030EDB2A66
:10120000040E01E3DB2AF05103E0020EF05D17E16A
:10121000020EE76E030EDBCFE9FF040EDBCFEAFF21
:10122000E750E926000EEA22C00EE926040EEA2263
:101230000A0EEF6E030EDB2A040E01E3DB2A030E17
:10124000DBCF25F0040EDBCF26F0020E25240401AF
:10125000C16FF90EDBCFC0F1FA0EDBCFC1F1186A16
:10126000DDEC1DF00A0EE66ECAEC23F0E5520CEC44
:101270001DF00CEC1DF0010E14141BE0080E1414EC
:1012800018E00401320EC06F050EC16F3F0EC26F31
:10129000550EC36F400E0501EF250401C46FC56BE9
:1012A000DDEC1DF00A0EE66EBCEC23F0E5520CEC12
:1012B0001DF0010EF36E070EF3CFDBFF080EDB6AA5
:1012C0003DD1F90EDB500101C05D256EFA0EDB50F9
:1012D000C1590001266ED890E85004E63D0E255C09
:1012E000000E265801E21FD114A61FD00401320EB1
:1012F000C06F050EC16F3F0EC26F550EC36F200E3B
:101300000501EF250401C46FC56BDDEC1DF00A0E6D
:10131000E66ECAEC23F0E5520CEC1DF0010EE66E11
:10132000DDEC1FF0E552DDEC1DF0030EDB6A040E70
:10133000DB6AF90EDBCF06F0FA0EDBCF07F00B0EFF
:1013400006C0DBFF0C0E07C0DBFF400EE66EE66A50
:10135000E66AC00EE66E040EE66EE0EC20F0256E46
:10136000050EE15E25500401200EC06F0B0EDBCF91
:1013700025F00C0EDBCF26F00101C051255CC151D8
:10138000265826E20B0EDBCFE9FF0C0EDBCFEAFF7F
:10139000EF50E66E020EE76E030EDBCFE9FF040EA0
:1013A000DBCFEAFFE750E926000EEA22C00EE9266D
:1013B000040EEA22E552E750EF6E0B0EDB2A0C0E0C
:1013C00001E3DB2A030EDB2A040ED0E3DB2ACED7AF
:1013D000030EDBCF25F0040EDBCF26F0020E252412
:1013E0000401C16FF90EDBCFC0F1FA0EDBCFC1F102
:1013F000186ADDEC1DF00A0EE66ECAEC23F0E55229
:101400000CEC1DF00CEC1DF0010EF36E070EF3CF8B
:10141000DBFF080EDB6A87D0DF50C0C1E9FFC1C126
:10142000EAFFEF6E0101C02B000EC123182A6DD018
:101430002B0EDF5C16E1030EEE6F320EE66EE66AEF
:10144000E66A400EE66E020EE66EE0EC20F0256ED7
:10145000050EE15E25500001400EFB6F020EFC6F91
:101460006DD0EE6B60D00D0EDF5C03E00A0EDF5C2A
:101470004FE1FBC0E9FFFCC0EAFFEF6AFBC025F0CB
:10148000FCC026F0400E255E020E265A25C0E6FF5F
:1014900026C0E6FFF50EDBCFE6FFF60EDBCFE6FF5C
:1014A000400EE66E020EE66E64D8276E060EE15E12
:1014B0002750DE52F3CFDEFFF4CFDDFFDD52D950EF
:1014C000010FE96EDACFEAFFEE50ED1014E10101F1
:1014D000C0C1E9FFC1C1EAFFC02B000EC1232B0E22
:1014E000EF6EC0C1E9FFC1C1EAFFC02B000EC123EE
:1014F0002B0EEF6E0AD0F50EDBCFE6FFF60EDBCF3C
:10150000E6FF8BEC1CF0E552E5520501EE6B16D0C0
:10151000DF50FBC0E9FFFCC0EAFFEF6E0001FB2BD0
:10152000000EFC230BD0DF50C0C1E9FFC1C1EAFFB0
:10153000EF6E0101C02B000EC123182A050EDB2A15
:10154000060E01E286D5DB2A84D5070EDBCF25F017
:10155000080EDBCF26F025C0F3FF26C0F4FF0D0EEA
:10156000E15C02E2E16AE552E16EE552E7CFD9FFC4
:101570001200D9CFE6FFE1CFD9FF530EE126F90ED5
:10158000DBCF25F0FA0EDBCF26F0263406E225501D
:101590003208000E265401E2D2D1FD0EDBCF06F058
:1015A000FE0EDBCF07F0DE5206C0DEFF07C0DDFF18
:1015B000DD52320EE66EE66AE66AD950050FE66E37
:1015C000000EDA20E66EE0EC20F0256E050EE15EFE
:1015D00025504B0EDB6A4C0EDB6A4B0EDBCF25F041
:1015E0004C0EDBCF26F0F90EDBCF27F0FA0EDBCF67
:1015F00028F026502818E8AE02D0283404D027500E
:10160000255C2850265829E2010EDBCFE9FFDB2AB2
:10161000020EDBCFEAFF01E3DB2AEFCFDFFF0D0E87
:10162000DF5C1BE00A0EDF5C18E0200EDF5C15E0DB
:10163000D950050F256EDACF26F04B0EDB5025244E
:10164000E96E4C0EDB50DA20EA6EDFCFEFFF4B0E77
:10165000DB2A4C0EC2E3DB2AC0D7D950030FE96E58
:10166000DACFEAFFE90EEE6E050EED6E200EDF5CBE
:1016700001E08DD04B0EDBCF25F0DB2A4C0EDBCF0B
:1016800026F001E3DB2AF90EDBCF27F0FA0EDBCFE1
:1016900028F026502818E8AE02D0283404D027506D
:1016A000255C2850265843E2010EDBCFE9FF020EED
:1016B000DBCFEAFFEFCFDFFF200EDF5CDBE0DFCF29
:1016C000E6FFE66A66EC23F0E552E552F3CF27F039
:1016D000F4CF28F0F3CFE6FFF4CFE6FFDFCFE6FF4D
:1016E000E66A7EEC23F0E552E552E552E7CF28F0BA
:1016F000E552E7CF27F02750F310256E2850F4105D
:10170000266E255026100DE0010EDBCF06F0020EEE
:10171000DBCF07F0030E06C0DBFF040E07C0DBFFC4
:1017200006D0010EDB2A020EA5E3DB2AA3D74B0E5F
:10173000DBCF25F0DB2A4C0EDBCF26F001E3DB2AE2
:10174000F90EDBCF27F0FA0EDBCF28F02650281851
:10175000E8AE02D0283404D02750255C2850265803
:1017600016E2010EDBCFE9FF020EDBCFEAFFEFCF7F
:10177000DFFF0D0EDF5C0BE00A0EDF5C08E0DF50E0
:1017800006E0010EDB2A020ED2E3DB2AD0D74B0E95
:10179000DBCF06F04C0EDBCF07F04F0E06C0DBFFB1
:1017A000500E07C0DBFF4B0EDB6A4C0EDB6A4B0EA4
:1017B000DBCF25F04C0EDBCF26F0D890265004E688
:1017C000640E255C000E265801E3B9D04B0EDBCF2A
:1017D000E9FF4C0EDBCFEAFFD890E936EA36D89025
:1017E000E936EA36910EE926050EEA22020EE926CE
:1017F000000EEA22EE50ED1001E1A1D04B0EDBCF3E
:10180000E9FF4C0EDBCFEAFFD890E936EA36D890F4
:10181000E936EA36910EE926050EEA22EECF25F0EA
:10182000EFCF26F0276A25C0E6FF26C0E6FF27C0D7
:10183000E6FFFAEC20F0E552E552E552510E05C004
:10184000DBFF520E06C0DBFF510EDBCFE6FF520E70
:10185000DBCFE6FFFD0EDBCFE6FFFE0EDBCFE6FFC4
:101860004B0EDBCFE9FF4C0EDBCFEAFFD890E93619
:10187000EA36D890E936EA36910EE926050EEA22D4
:10188000EECF25F0EFCF26F0276A25C0E6FF26C071
:10189000E6FF27C0E6FF1FEC21F0286E070EE15E91
:1018A0002850000945E14B0EDBCFE9FF4C0EDBCFA2
:1018B000EAFFD890E936EA36D890E936EA36910E52
:1018C000E926050EEA22020EE926000EEA22EECFF4
:1018D00025F0EFCF26F0030EDBCFE6FF040EDBCFC3
:1018E000E6FFFB0EDBCFE6FFFC0EDBCFE6FFFD0ED7
:1018F000DBCFE6FFFE0EDBCFE6FF04D026C0FAFF0B
:101900002550F96EFBDF276E060EE15E27504D0E67
:10191000F3CFDBFF4E0EF4CFDBFF4F0EDBCF25F016
:10192000500EDBCF26F025C0F3FF26C0F4FF09D010
:101930004B0EDB2A4C0E01E23AD7DB2A38D7F36A8A
:10194000F46A530EE15C02E2E16AE552E16EE552AF
:10195000E7CFD9FF1200D9CFE6FFE1CFD9FFF90ECB
:10196000DBCF25F0FA0EDBCF26F0E90E25181EE1BD
:10197000050E26181BE10501EF51E66EE66A670EBB
:10198000256E400E266E276A25C0E6FFE66E27C04C
:10199000E6FFFB0EDBCFE6FFFC0EDBCFE6FF1AEC2B
:1019A00022F0286E070EE15E285013D0F90EDBCF2F
:1019B000E6FFFA0EDBCFE6FF6BEC20F0E552E552D6
:1019C000F3CFEFF5FB0EDBCFE9FFFC0EDBCFEAFF39
:1019D000EF6A010EF36EF46AE552E7CFD9FF120009
:1019E000D9CFE6FFE1CFD9FF020EE126DE6ADD6A3C
:1019F000F90EDBCF25F0FA0EDBCF26F0E90E251825
:101A00002CE1050E261829E1010E141402E1000E46
:101A100001D0010E256E266A25BE266825C0DEFF90
:101A200026C0DDFFDECFE6FFDDCFE6FF670E256EC9
:101A3000400E266E276A25C0E6FFE66E27C0E6FF49
:101A4000FB0EDBCFE6FFFC0EDBCFE6FF1AEC22F04D
:101A5000286E070EE15E285024D0F90EDBCFE6FF9A
:101A6000FA0EDBCFE6FF6BEC20F0E552E552F3CF48
:101A7000DEFFF4CFDDFFD9CFE9FFDACFEAFF010EB9
:101A8000EE1805E1ED5003E1010E141002D0FE0E38
:101A90001414146EFB0EDBCFE9FFFC0EDBCFEAFF64
:101AA000EF6A010EF36EF46A020EE15C02E2E16A93
:101AB000E552E16EE552E7CFD9FF1200D9CFE6FF3C
:101AC000E1CFD9FF410E256E400E266E276A25C054
:101AD000E6FFE66E27C0E6FFFB0EDBCFE6FFFC0E5F
:101AE000DBCFE6FF1AEC22F0286E050EE15E2850EF
:101AF000010EF36EF46AE552E7CFD9FF1200D9CF99
:101B0000E6FFE1CFD9FFB4EC1FF0FB0EDBCFE9FF1E
:101B1000FC0EDBCFEAFFEF6A010EF36EF46AE552CA
:101B2000E7CFD9FF1200D9CFE6FFE1CFD9FF070EEB
:101B3000E66E400EE66E130E256E400E266E276A88
:101B400025C0E6FFE66E27C0E6FFFB0EDBCFE6FF13
:101B5000FC0EDBCFE6FF1AEC22F0286E070EE15EEA
:101B60002850010EF36EF46AE552E7CFD9FF120058
:101B7000D9CFE6FFE1CFD9FF0401320EC06F060EC8
:101B8000C16F3F0EC26F550EC36F200E0501EF25CA
:101B90000401C46F040EC56FC66BDDEC1DF0FB0EB7
:101BA000DBCFE9FFFC0EDBCFEAFFEF6A010EF36E3D
:101BB000F46AE552E7CFD9FF1200D9CFE6FFE1CFB3
:101BC000D9FF020EE126DE6ADD6AF90EDBCF25F0D1
:101BD000FA0EDBCF26F0E90E25182CE1050E2618AB
:101BE00029E1020E141402E1000E01D0010E256E4F
:101BF000266A25BE266825C0DEFF26C0DDFFDECFB3
:101C0000E6FFDDCFE6FF670E256E400E266E276AE3
:101C100025C0E6FFE66E27C0E6FFFB0EDBCFE6FF42
:101C2000FC0EDBCFE6FF1AEC22F0286E070EE15E19
:101C3000285024D0F90EDBCFE6FFFA0EDBCFE6FF0B
:101C40006BEC20F0E552E552F3CFDEFFF4CFDDFF81
:101C5000D9CFE9FFDACFEAFF010EEE1805E1ED502A
:101C600003E1020E141002D0FD0E1414146EFB0ECC
:101C7000DBCFE9FFFC0EDBCFEAFFEF6A010EF36E6C
:101C8000F46A020EE15C02E2E16AE552E16EE552BD
:101C9000E7CFD9FF1200D9CFE6FFE1CFD9FFF90E88
:101CA000DBCF25F0FA0EDBCF26F0E90E25181EE17A
:101CB000050E26181BE10501F051E66EE66A670E77
:101CC000256E400E266E276A25C0E6FFE66E27C009
:101CD000E6FFFB0EDBCFE6FFFC0EDBCFE6FF1AECE8
:101CE00022F0286E070EE15E285013D0F90EDBCFEC
:101CF000E6FFFA0EDBCFE6FF6BEC20F0E552E55293
:101D0000F3CFF0F5FB0EDBCFE9FFFC0EDBCFEAFFF4
:101D1000EF6A010EF36EF46AE552E7CFD9FF1200C5
:101D2000D9CFE6FFE1CFD9FF020EE126DE6ADD6AF8
:101D3000F90EDBCF25F0FA0EDBCF26F0E90E2518E1
:101D40002CE1050E261829E1040E141402E1000E00
:101D500001D0010E256E266A25BE266825C0DEFF4D
:101D600026C0DDFFDECFE6FFDDCFE6FF670E256E86
:101D7000400E266E276A25C0E6FFE66E27C0E6FF06
:101D8000FB0EDBCFE6FFFC0EDBCFE6FF1AEC22F00A
:101D9000286E070EE15E285024D0F90EDBCFE6FF57
:101DA000FA0EDBCFE6FF6BEC20F0E552E552F3CF05
:101DB000DEFFF4CFDDFFD9CFE9FFDACFEAFF010E76
:101DC000EE1805E1ED5003E1040E141002D0FB0EF5
:101DD0001414146EFB0EDBCFE9FFFC0EDBCFEAFF21
:101DE000EF6A010EF36EF46A020EE15C02E2E16A50
:101DF000E552E16EE552E7CFD9FF1200D9CFE6FFF9
:101E0000E1CFD9FFF90EDBCF25F0FA0EDBCF26F0BC
:101E1000E90E25181EE1050E26181BE10501F151FA
:101E2000E66EE66A670E256E400E266E276A25C0AE
:101E3000E6FFE66E27C0E6FFFB0EDBCFE6FFFC0EFB
:101E4000DBCFE6FF1AEC22F0286E070EE15E285089
:101E500013D0F90EDBCFE6FFFA0EDBCFE6FF6BEC1B
:101E600020F0E552E552F3CFF1F5FB0EDBCFE9FFB1
:101E7000FC0EDBCFEAFFEF6A010EF36EF46AE55267
:101E8000E7CFD9FF1200D9CFE6FFE1CFD9FFE66A4D
:101E9000DDEC1FF0E552FB0EDBCFE9FFFC0EDBCFE4
:101EA000EAFFEF6A010EF36EF46AE552E7CFD9FF5D
:101EB0001200D9CFE6FFE1CFD9FF020EE126DE6A9C
:101EC000DD6AF90EDBCF25F0FA0EDBCF26F0E90E46
:101ED00025182CE1050E261829E1100E141402E134
:101EE000000E01D0010E256E266A25BE266825C08B
:101EF000DEFF26C0DDFFDECFE6FFDDCFE6FF670EAB
:101F0000256E400E266E276A25C0E6FFE66E27C0C6
:101F1000E6FFFB0EDBCFE6FFFC0EDBCFE6FF1AECA5
:101F200022F0286E070EE15E285024D0F90EDBCF98
:101F3000E6FFFA0EDBCFE6FF6BEC20F0E552E55250
:101F4000F3CFDEFFF4CFDDFFD9CFE9FFDACFEAFF31
:101F5000010EEE1805E1ED5003E1100E141002D051
:101F6000EF0E1414146EFB0EDBCFE9FFFC0EDBCF7B
:101F7000EAFFEF6A010EF36EF46A020EE15C02E220
:101F8000E16AE552E16EE552E7CFD9FF1200D9CF01
:101F9000E6FFE1CFD9FF020EE126DE6ADD6AF90E27
:101FA000DBCF25F0FA0EDBCF26F0E90E25182CE169
:101FB000050E261829E1080E141402E1000E01D0C6
:101FC000010E256E266A25BE266825C0DEFF26C0C6
:101FD000DDFFDECFE6FFDDCFE6FF670E256E400EAC
:101FE000266E276A25C0E6FFE66E27C0E6FFFB0ED9
:101FF000DBCFE6FFFC0EDBCFE6FF1AEC22F0286E0B
:10200000070EE15E285029D0F90EDBCFE6FFFA0E6D
:10201000DBCFE6FF6BEC20F0E552E552F3CFDEFFBD
:10202000F4CFDDFFD9CFE9FFDACFEAFF010EEE18DA
:1020300006E1ED5004E1080E1410146E07D0F70EFF
:102040001414146EE66ADDEC1FF0E552FB0EDBCFD4
:10205000E9FFFC0EDBCFEAFFEF6A010EF36EF46AD4
:10206000020EE15C02E2E16AE552E16EE552E7CF81
:10207000D9FF1200D9CFE6FFE1CFD9FFF90EDBCFB0
:1020800025F0FA0EDBCF26F0E90E251806E1050E45
:10209000261803E10501F46B31D0030EE66EE66A03
:1020A000F90EDBCFE6FFFA0EDBCFE6FFC40E256E9E
:1020B000400E266E276A25C0E6FFE66E27C0E6FFC3
:1020C0001FEC21F0286E070EE15E2850000903E1A5
:1020D0000501010E12D0F90EDBCFE6FFFA0EDBCFC1
:1020E000E6FF6BEC20F0E552E552F3CFE7F101019A
:1020F000E751000803E20501020EF46F0401320EFD
:10210000C06F050EC16F3F0EC26F550EC36F400EFC
:102110000501EF250401C46FC56BDDEC1DF0FB0E5E
:10212000DBCFE9FFFC0EDBCFEAFFEF6A010EF36EB7
:10213000F46AE552E7CFD9FF1200D9CFE6FFE1CF2D
:10214000D9FFF90EDBCF25F0FA0EDBCF26F0E90E32
:1021500025181EE1050E26181BE1F2C5E6FFF3C5A2
:10216000E6FF670E256E400E266E276A25C0E6FF45
:10217000E66E27C0E6FFFB0EDBCFE6FFFC0EDBCFF3
:10218000E6FF1AEC22F0286E070EE15E285015D00B
:10219000F90EDBCFE6FFFA0EDBCFE6FF6BEC20F0AB
:1021A000E552E552F3CFF2F5F4CFF3F5FB0EDBCFBA
:1021B000E9FFFC0EDBCFEAFFEF6A010EF36EF46A73
:1021C000E552E7CFD9FF1200D9CFE6FFE1CFD9FF23
:1021D000400EE66EE66AE66A800EE66E010EE66E78
:1021E000E0EC20F0256E050EE15E25500501EE6B5A
:1021F000090E146E0501F06B05012A0EF16F050141
:102200002C0EF26F010EF36F0501F46FD950FB0F26
:10221000E96EDACFEAFF800EEE6E010EED6E176A00
:10222000186A010EF36EF46AE552E7CFD9FF120087
:10223000D9CFE6FFE1CFD9FF020EE1260501EF512C
:10224000DE6EDD6AFB0EDBCFE9FFFC0EDBCFEAFFC3
:10225000EF6AF90EDBCF25F0FA0EDBCF26F0E90EA0
:10226000251802E1050E26180EE0F90EDBCFE6FF79
:10227000FA0EDBCFE6FF6BEC20F0E552E552F3CF30
:10228000DEFFF4CFDDFF0401320EC06F060EC16F1A
:102290003F0EC26F350EC36F180EC46FDECF25F030
:1022A000DDCF26F0400E2524C56FDDEC1DF0B6EC29
:1022B0001EF0175000081BE204014051E66EE66A6A
:1022C000670E256E400E266E276A25C0E6FFE66E75
:1022D00027C0E6FFFB0EDBCFE6FFFC0EDBCFE6FF01
:1022E0001AEC22F0286E070EE15E2850176A0401EE
:1022F000320EC06F050EC16F190EC26F5F0EC36F35
:102300003F0EC46FC56BDDEC1DF0010EF36EF46A79
:10231000020EE15C02E2E16AE552E16EE552E7CFCE
:10232000D9FF1200D9CFE6FFE1CFD9FF020EE12697
:10233000010EDE6EDD6A80A402D0DE6ADD6ADECFC9
:10234000E6FFDDCFE6FF670E256E400E266E276A9C
:1023500025C0E6FFE66E27C0E6FFFB0EDBCFE6FFFB
:10236000FC0EDBCFE6FF1AEC22F0286E070EE15ED2
:102370002850010EF36EF46A020EE15C02E2E16A9B
:10238000E552E16EE552E7CFD9FF1200D9CFE6FF63
:10239000E1CFD9FF020EE1260501EF51DE6EDD6AC5
:1023A000FB0EDBCFE9FFFC0EDBCFEAFFEF6AF90E95
:1023B000DBCF25F0FA0EDBCF26F0E90E251802E17F
:1023C000050E26180EE0F90EDBCFE6FFFA0EDBCF86
:1023D000E6FF6BEC20F0E552E552F3CFDEFFF4CFE1
:1023E000DDFF0401320EC06F060EC16F3F0EC26FDB
:1023F000550EC36FDECF25F0DDCF26F0200E25244D
:10240000C46F080EC56FC66BDDEC1DF0010EF36ED8
:10241000F46A020EE15C02E2E16AE552E16EE55225
:10242000E7CFD9FF1200D9CFE6FFE1CFD9FFFB0EEE
:10243000DBCFE9FFFC0EDBCFEAFFEF6A010EF36EA4
:0A244000F46AE552E7CFD9FF12005D
:06244A00D9CFE6FFE1CF4F
:10245000D9FFE652A09A6A6A686A706A020EE66E4E
:10246000E66AE66A710EE66E0F0EE66EE0EC20F0AC
:10247000256E050EE15E2550160E6F6E9F0E6B6E7B
:102480007B0E696EDF6ADF50256E266A0C0E255CB6
:10249000000E265810E2DF50040DF3CFE9FFF4CF11
:1024A000EAFF000EE926040EEA22EE6AEE6AEE6A00
:1024B000EE6ADF2AE8D76D8C6E6A6D986D9C68A60F
:1024C00007D0689602018A6B8F6B906B916BF7D780
:1024D0000201010EA36FA46FA56BA66B976BDF6A59
:1024E000030EDF5C26E2EA6ADF34FE0BEA36E96EB1
:1024F000800EE926020EEA22EE6AED6AEA6ADF340D
:10250000FE0BEA36E96E7A0EE926020EEA22EE6A40
:10251000ED6ADF50EA6A9B0FE96E020EEA22EF6A6B
:10252000DF50EA6A9E0FE96E020EEA22EF6ADF2AA6
:10253000D7D70201080E806F040E816F160E706EE1
:102540000401300E026F040E036F080E016F840E3B
:10255000006F0201736B726BE552E552E7CFD9FF52
:102560001200D9CFE6FFE1CFD9FFE6520201725146
:102570000FE16D6A696A160E6F6E9F0E6B6E7B0EB1
:10258000696E6DB602D06D86FCD70201010E726FC6
:10259000720508E16DBA06D0686A696A698069885F
:1025A000020E726F6850040B06E06950040B03E0E2
:1025B00068948CEC18F06DB258D06850010B08E0AC
:1025C0006950010B05E041DF0201040E726F689053
:1025D0006850100B06E06950100B03E077EC18F020
:1025E000689868AC19D069AC0FD0010EE66EE66A47
:1025F000000EE66EE66A730EE66EE66A0DEC07F014
:10260000256E060EE15E2550689C0201A15101E095
:10261000A107A15101E1DFD96850200B05E0695005
:10262000200B02E05EEC18F06850020B13E06950DA
:10263000020B10E0010EE66EE66A000EE66EE66A38
:10264000E6687F0EE66E0DEC07F0256E060EE15E85
:1026500025506A6A040E0201E76E7219E8AE02D0D4
:10266000E73402D0E750725D02E2A19A39D069A640
:1026700036D0DF6A040EDF5C32E268A630D06CCF61
:1026800098F202019851780BE842E842E842996FCB
:10269000689698B506D09951EA6A9E0FE96E020EC7
:1026A00005D09951EA6A9B0FE96E020EEA22EF709B
:1026B000995103E1A3EC18F010D0000EE66EE66A23
:1026C000980EE66E020EE66E720EE66EE66A0DEC8F
:1026D00007F0256E060EE15E2550DF2ACBD7A19AC2
:1026E000E552E552E7CFD9FF1200D9CFE6FFE1CF9F
:1026F000D9FF020EE126FD0EDBA407D0E66AFE0E2E
:10270000DBCFE6FFF7D9E552E552FD0EDBA208D09C
:10271000010EE66EFE0EDBCFE6FFECD9E552E55288
:10272000FE0EDB50266A700F256E0F0E262225C086
:10273000DEFF26C0DDFFDECFE9FFDDCFEAFFFD0EC5
:10274000DBCFEFFF020EE15C02E2E16AE552E16EEF
:10275000E552E7CFD9FF1200D9CFE6FFE1CFD9FF8D
:10276000020EE126FD0EDB500AE0FE0EEA6ADB34C3
:10277000FE0BEA36E96E800EE926020E09D0FE0E47
:10278000EA6ADB34FE0BEA36E96E7A0EE926020EBF
:10279000EA22EECFDEFFEDCFDDFFD9CFE9FFDACFC2
:1027A000EAFFEE50ED1003E1F36AF46A44D0DECFA5
:1027B000E9FFDDCFEAFF020EE926000EEA22FB0E5A
:1027C000DBCFEEFFFC0EDBCFEDFFDECFE9FFDDCF91
:1027D000EAFFEE52FA0EDBCFEFFF400EDECFE9FF4D
:1027E000DDCFEAFFE850EF16880EDECFE9FFDDCF40
:1027F000EAFFE850EF12FD0EDB500AE0FE0EEA6A37
:10280000DB34FE0BEA36E96E800EE926020E09D0B3
:10281000FE0EEA6ADB34FE0BEA36E96E7A0EE92632
:10282000020EEA22EF74DECF25F0DDCF26F025C0C0
:10283000F3FF26C0F4FF020EE15C02E2E16AE5521A
:10284000E16EE552E7CFD9FF1200D9CFE6FFE1CF25
:10285000D9FF020EE126FE0EDB5020E178C2E9FF2F
:1028600079C2EAFFEE52080EEF6E78C2E9FF79C234
:10287000EAFF020EE926000EEA22300EEE6E040E8A
:10288000ED6E78C2E9FF79C2EAFF8C0EEF6E80C26E
:10289000E9FF81C2EAFF840EEF6E3BD0FD0EDB50F4
:1028A000E824276EFE0EDB50040DF3502724040DA0
:1028B000F3CF25F0F4CF26F0000E2526040E2622B5
:1028C00025C0DEFF26C0DDFF840EDECFE9FFDDCFB1
:1028D000EAFFE850EF12FD0EDB50E824276EFE0EF3
:1028E000DB50040DF3502724010F040DF3CF25F026
:1028F000F4CF26F0000E2526040E262225C0DEFF8A
:1029000026C0DDFF840EDECFE9FFDDCFEAFFE85011
:10291000EF12020EE15C02E2E16AE552E16EE5527D
:10292000E7CFD9FF1200D9CFE6FFE1CFD9FF6DA8DD
:102930004ED0FE0EEA6ADB34FE0BEA36E96E800EFC
:10294000E926020EEA22EE50EFCFEAFFE96E400ED2
:10295000EE16EE6AEE6AEE6AFE0EEA6ADB34FE0BF3
:10296000EA36E96E800EE926020EEA22EE50EFCF3B
:10297000EAFFE96EEE7CFE0EEA6ADB34FE0BEA3615
:10298000E96E800EE926020EEA22EF74400E256EF3
:10299000FE0EEA6ADB34FE0BEA36E96E800EE926AB
:1029A000020EEA22EE50EFCFEAFFE96E2550EF1655
:1029B000FE0EEA6ADB34FE0BEA36E96E800EE9268B
:1029C000020EEA22EE50EFCFEAFFE96EEF7CE5520D
:1029D000E7CFD9FF12000201A3514DE1010EA36F11
:1029E000A45149E1010EA46F020E875D0DE180C282
:1029F000E9FF81C2EAFFEE52EF6A80C2E9FF81C2BD
:102A0000EAFFC80EEF6E1200870535E19A6B76C2B9
:102A1000E9FF77C2EAFFEE52080EEF6E76C2E9FFD9
:102A200077C2EAFF020EE926000EEA22300EEE6EB1
:102A3000040EED6E76C2E9FF77C2EAFF840EEF6EF8
:102A4000010E9A6F78C2E9FF79C2EAFFEE52080ED2
:102A5000EF6E78C2E9FF79C2EAFF020EE926000EA6
:102A6000EA22300EEE6E040EED6E78C2E9FF79C2F6
:102A7000EAFF800EEF6E12000201A56BA66B020E3C
:102A8000875D18E178C2E9FF79C2EAFFEE52080ECD
:102A9000EF6E78C2E9FF79C2EAFF020EE926000E66
:102AA000EA22380EEE6E040EED6E78C2E9FF79C2AE
:102AB000EAFF1DD08B510401365D02018C510401E7
:102AC000375904E236C48BF237C48CF2CAD880C2BC
:102AD000E9FF81C2EAFF020EE926000EEA22380E63
:102AE000EE6E040EED6E80C2E9FF81C2EAFFC80EF1
:102AF000EF6E1200D9CFE6FFE1CFD9FF020EE1263B
:102B0000000EDE6E040EDD6EFD0EDB50E824276E37
:102B1000FE0EDB50040DF3502724040DF4CF26F0F5
:102B2000D9CFE9FFDACFEAFFF350EE262650ED22A7
:102B3000DECFE9FFDDCFEAFFEF9EFD0EDB500AE1BD
:102B4000FE0EEA6ADB34FE0BEA36E96E7A0EE926FF
:102B5000020E09D0FE0EEA6ADB34FE0BEA36E96E9D
:102B6000800EE926020EEA22DECFEEFFDDCFEDFF7A
:102B7000DECFE9FFDDCFEAFFEF9CDECFE9FFDDCF5F
:102B8000EAFF040EE926000EEA22EF8C020EE15C59
:102B900002E2E16AE552E16EE552E7CFD9FF1200A9
:102BA0006D9802018ABF2BD08FAF09D0020E876FBC
:102BB000A65101E161DF0201A46BA36B120078C290
:102BC000E9FF79C2EAFFEE52080EEF6E78C2E9FF24
:102BD00079C2EAFF020EE926000EEA22300EEE6EFE
:102BE000040EED6E78C2E9FF79C2EAFF8C0EEF6E3B
:102BF00080C2E9FF81C2EAFF840EEF6E1200040179
:102C000030AF0DD00201010E876FA55101E134DF15
:102C10000201A46BA36BA25123E1EBEF14F00201BC
:102C2000020E876F78C2E9FF79C2EAFFEE52080E02
:102C3000EF6E78C2E9FF79C2EAFF020EE926000EC4
:102C4000EA22300EEE6E040EED6E78C2E9FF79C214
:102C5000EAFF840EEF6EA46BA36BA25101E1BBDE11
:102C60001200D9CFE6FFE1CFD9FFE652080EDF6EA2
:102C700002018B5D000E8C590AE28BC2DFFF865188
:102C800002E1010E03D0860502E1020E866FDF50DD
:102C9000266AE8508B5D8B6F26508C598C6F80C2F2
:102CA000E9FF81C2EAFFEE52DFCFEFFF380E946FEB
:102CB000040E956F8AB118D0DF502DE088C2F6FF60
:102CC00089C2F7FF882B000E89230800F550E66EB5
:102CD00094C2E9FF95C2EAFF942B000E9523E552BA
:102CE000E750EF6EDF06E8D7DF5015E088C2E9FF56
:102CF00089C2EAFF882B000E8923EF50E66E94C24A
:102D0000E9FF95C2EAFF942B000E9523E552E750A8
:102D1000EF6EDF06E9D7E552E552E7CFD9FF1200A3
:102D2000D9CFE6FFE1CFD9FF020EE12676C2E9FF57
:102D300077C2EAFFEE52EFCFDFFFDFCF25F025505D
:102D40000201905D000E915902E290C2DFFFDF5058
:102D5000256E266AE850905D906F26509159916FCC
:102D6000010EDB6ADF50F36E010EDBCFF4FFF35090
:102D7000F45C16E2010EDB50EA6A380FE96E040ECD
:102D8000EA22EF50E66E8DC2E9FF8EC2EAFF8D2B7C
:102D9000000E8E23E552E750EF6E010EDB2AE2D7DC
:102DA000000ED8809055000E915527E278C2E9FFB9
:102DB00079C2EAFFEE52080EEF6E78C2E9FF79C2DF
:102DC000EAFF020EE926000EEA22380EEE6E040E2D
:102DD000ED6E76C2E9FF77C2EAFFEF50400B06E1E5
:102DE00078C2E9FF79C2EAFFC80E05D078C2E9FFD0
:102DF00079C2EAFF880EEF6E28D078C2E9FF79C267
:102E0000EAFFEE52080EEF6E78C2E9FF79C2EAFFE0
:102E1000020EE926000EEA22300EEE6E040EED6E72
:102E200078C2E9FF79C2EAFF840EEF6E92519311E6
:102E300007E005D093C2FAFF02019251F96EFADF62
:102E400002018F9FA25101E1C6DD020EE15C02E2A8
:102E5000E16AE552E16EE552E7CFD9FF1200D9CF22
:102E6000E6FFE1CFD9FFE65202018A8F020EE66E3D
:102E7000E66AE66A710EE66E0F0EE66EE0EC20F092
:102E8000256E050EE15E2550300EE66EE66AE66AB6
:102E9000000EE66E040EE66EE0EC20F0256E050EE8
:102EA000E15E25506D8CDF6A030EDF5C10E2DF50BF
:102EB000EA6A9B0FE96E020EEA22EF6ADF50EA6AC5
:102EC0009E0FE96E020EEA22EF6ADF2AEDD7020EAC
:102ED000E66EE66AE66A740EE66E020EE66EE0ECF8
:102EE00020F0256E050EE15E25506D9C0201080E56
:102EF000806F040E816F000E766F040E776F76C2BE
:102F000078F2796F32C473F2735102E1100E12D06D
:102F1000010EE66EE66A730EE66E020EE66E010EB6
:102F2000E66EE66A0DEC07F0256E060EE15E2550B2
:102F30000201200E726FE552E552E7CFD9FF120071
:102F4000800E0401305D58E10201C00E8A6F040159
:102F50003351030A2FE0010A09E0030A4BE10201A1
:102F60006A0E886F430E896F120E3ED03251F66E94
:102F7000F76AD890F636F7362B0EF626440EF7226F
:102F80000900F5CF88F20A00F5CF89F2020E02019E
:102F9000F76A8825F66E8951F7220800F5CF8BF283
:102FA000030EF76A8825F66E8951F7220800F5CFDF
:102FB0008CF21200030E325D1AE23251F66EF76A9D
:102FC000D890F636F7362D0EF626440EF722090075
:102FD000F5CF88F20A00F5CF89F288C2F6FF89C2E0
:102FE000F7FF0800F55002018B6F8C6B1200020195
:102FF0008A6B120002018A6B1200D9CFE6FFE1CF83
:10300000D9FF020EE1260401386B396B30511F0BDA
:10301000020A11E0030A0CE0010A3CE102018A8F76
:10302000040138810201960535E10401388332D06C
:1030300002018A8F2FD002018A8F040134BF0BD086
:1030400034510F0BE96EEA6AD890E936EA367A0E07
:10305000E926020E0AD034510F0BE96EEA6AD890C5
:10306000E936EA36800EE926020EEA22EECFDEFFCE
:10307000EDCFDDFFDECFE9FFDDCFEAFFEF50800BC4
:1030800009E0DECFE9FFDDCFEAFFEF50040B02E0FD
:10309000010E386F02018AAF07D0380E886F040E18
:1030A000896F8A81020E8B6F020EE15C02E2E16A97
:1030B000E552E16EE552E7CFD9FF120070A015D0BE
:1030C00076C2E9FF77C2EAFFEF5080080DE180C2C7
:1030D000E9FF81C2EAFFEF50840806E176C2E9FF0A
:1030E00077C2EAFF8C0EEF6E7090689A12006984C6
:1030F00068986D820201010E976F000EE66EE66A17
:10310000E66EE66A750EE66EE66A0DEC07F0256E71
:10311000060EE15E255012000201976B000EE66E6E
:10312000E66AE66EE66A740EE66EE66A0DEC07F095
:10313000256E060EE15E25506D92699468A402D05A
:103140006894FCD71200D9CFE6FFE1CFD9FFE65251
:1031500002012D0EA16FFD0E981553E17E0E9815FC
:10316000E8407F0B040DF3CF76F2F4CF77F2000E38
:103170007627040E772376C278F277C279F27875D3
:1031800076C2E9FF77C2EAFFEF503C0BE842E84223
:103190000D0835E1DF6A080EDF5C23E276C2E9FF45
:1031A00077C2EAFF020EE926000EEA22EE50EFCFC8
:1031B000EAFFE96EEF50E66EDF50EA6A300FE96E23
:1031C000040EEA22E552E750EF6E76C2E9FF77C2BD
:1031D000EAFF020EE926000EEA22EE2AEF22DF2A9B
:1031E000DAD776C2E9FF77C2EAFF020EE926000EBF
:1031F000EA22300EEE6E040EED6E0DD807D03AD8EE
:1032000005D0FD0E9815040801E159D8E552E552A4
:10321000E7CFD9FF12000201866BA26BA56BA66BEC
:103220009A6B876B80C2E9FF81C2EAFFEF9E8075CF
:1032300080C2E9FF81C2EAFFEF9E807578C2E9FF94
:1032400079C2EAFFEF9E8A6B8B6B8C6B8F6B906BF6
:10325000916B8CD8000EE66EE66AE66EE66A030EA7
:10326000E66EE66A0DEC07F0256E060EE15E25506F
:10327000D0EF15F0020E0201875D02E190EF16F02B
:10328000876B9A511AE178C2E9FF79C2EAFFEE52E0
:10329000080EEF6E78C2E9FF79C2EAFF020EE92656
:1032A000000EEA22300EEE6E040EED6E78C2E9FFDB
:1032B00079C2EAFF8C0EEF6E12009A6B1200D9CF22
:1032C000E6FFE1CFD9FFE65280C2E9FF81C2EAFF03
:1032D000EF50400B01E0010EDF6E02018075080E19
:1032E000725D08E132C46EFF6E5002E0100E01D034
:1032F000040E726F870526E180C2E9FF81C2EAFFF2
:10330000020EE926000EEA22380EEE6E040EED6E75
:10331000A8DC020E0201865D06E180C2E9FF81C2DF
:10332000EAFF840E0DD0DF5006E180C2E9FF81C2C2
:10333000EAFFC80E05D080C2E9FF81C2EAFF880E0D
:10334000EF6E0FD08FAF0CD09251931107E005D0E4
:1033500093C2FAFF02019251F96EFADF02018F9FC8
:10336000876BE552E552E7CFD9FF120004013051D7
:10337000600BE842E842E842E842E842000901E026
:10338000120031510C0A50E00B0A3FE00C0A31E008
:10339000010A22E00B0A1EE0020A1CE0030A18E000
:1033A000080A10E0010A0CE00F0A08E0030A01E035
:1033B000120002018A8F080E726F1200A0EF17F040
:1033C0002FEF17F00201730E886F020E896F0CD079
:1033D000FDEF17F015EF1AF034510201886F896B79
:1033E000740E8827020E89238A81010E8B6F8A8FC3
:1033F000120002018A8F04013451EA6A740FE96EE7
:10340000020EEA2232C4EFFF1200000EE66EE66AF8
:10341000E66EE66A020EE66EE66A0DEC07F0256ED1
:10342000060EE15E255012001200D9CFE6FFE1CF73
:10343000D9FF050EE1260401320510E130511F0BC2
:1034400000090CE102018A8F030E0401315D04E1E1
:103450000201010E966F02D00201966B04013251F7
:1034600001E011D130511F0B020801E00CD13451A1
:103470000F0B000901E107D134510F0B020801E2E3
:1034800002D1200E0201725D01E0FDD08A8F04019D
:1034900034BF16D034510F0BE96EEA6AD890E93682
:1034A000EA367A0EE926020EEA22EECFDEFFEDCFF3
:1034B000DDFF34510F0BEA6A9E0FE96E020E15D044
:1034C00034510F0BE96EEA6AD890E936EA36800E7D
:1034D000E926020EEA22EECFDEFFEDCFDDFF34510A
:1034E0000F0BEA6A9B0FE96E020EEA22020EEFCF83
:1034F000DBFFD950020FE96EDACFEAFFEF50010B84
:1035000003E1000EDF9401D0DF8434BF0BD03451CF
:103510000F0BE96EEA6AD890E936EA367A0EE926A8
:10352000020E0AD034510F0BE96EEA6AD890E936E0
:10353000EA36800EE926020EEA22DECFEEFFDDCF6C
:10354000EDFF030E315D20E1DECFE9FFDDCFEAFFC5
:10355000EF50800B11E034BF07D034510F0BEA6AF3
:103560009E0FE96E020E06D034510F0BEA6A9B0FD4
:10357000E96E020EEA22EF82840EDECFE9FFDDCF94
:10358000EAFFE850EF127FD0DF74DECFE9FFDDCF36
:10359000EAFFEF50800B1BE0DECFE9FFDDCFEAFF53
:1035A000EF9EDECFE9FFDDCFEAFFEF8C020EE66E85
:1035B000E66ADECFE6FFDDCFE6FF050EE66EE66AE1
:1035C0000DEC07F0256E060EE15E255005D0DECF2E
:1035D000E9FFDDCFEAFFEF8CDF74D950020FE96E0F
:1035E000DACFEAFFEF50020B07E1DECFE9FFDDCFD4
:1035F000EAFFEF50800B2BE0040134BF07D03451B9
:103600000F0BEA6A9E0FE96E020E06D034510F0BC3
:10361000EA6A9B0FE96E020EEA22EF923B0E256EDC
:10362000DECFE9FFDDCFEAFFE850EF16020EE66ECF
:10363000E66ADECFE6FFDDCFE6FF050EE66EE66A60
:103640000DEC07F0256E060EE15E255007D03B0E0F
:10365000DECFE9FFDDCFEAFFE850EF160401345179
:103660000F0B266A700F256E0F0E2622030E25C043
:10367000DBFF040E26C0DBFF030EDBCFE9FF040EE9
:10368000DBCFEAFFEF90050EE15C02E2E16AE55272
:0A369000E16EE552E7CFD9FF12000A
:06369A00040130511F0B7A
:1036A000010801E012003051600BE842E842E842B4
:1036B000E842E842010801E01200345103E0340519
:1036C00001E012003151220A31E0030A24E0010A2C
:1036D00015E0210A0DE0010A01E012000201F30EDB
:1036E000886F000E896F080E8B6F8C6B8A8121D0DA
:1036F0000201F30E886F000E896F1BD036C490F262
:1037000037C491F20201800E8D6F050E8E6F926BA1
:10371000936B8F8F12000201800E886F050E896FE8
:10372000070E8B6F8C6BC10E8A6F120032C4EEF0E5
:1037300002018A8F12000501806B4B0E816F826B34
:10374000836B846B856B080E866F0001E26B1A0E2B
:10375000E66E010EE66E75EC13F0E552E5521E0EB4
:10376000E66E020EE66E75EC13F0E552E552400E81
:10377000E66E400EE66E050EE66EE66A020EE66E38
:10378000ACEC13F0256E050EE15E2550F3CFEAF0A8
:10379000F4CFEBF00001EC6BED6BE36B1200D9CFD3
:1037A000E6FFE1CFD9FFFD0EDBCF06F0FE0EDBCF4B
:1037B00007F0050E061801E1075002E0000E30D0B8
:1037C000FB0EDBCF25F0FC0EDBCF26F00001EA512B
:1037D000251816E1EB51261813E1400EE66E400E57
:1037E000E66E050EE66EE66A020EE66EACEC13F0CF
:1037F000256E050EE15E2550F3CFEAF0F4CFEBF035
:10380000FB0EDBCF25F0FC0EDBCF26F00001EC51E8
:10381000251805E1ED51261802E1E36BE86B010E76
:10382000E552E7CFD9FF1200D9CFE6FFE1CFD9FFAC
:103830000001E26BEA51EB1102E1000E08D0EAC090
:10384000E9FFEBC0EAFFEF50800B01E0010E000939
:1038500045E1FC0EDBCF25F0EAC0E9FFEBC0EAFF53
:10386000EE52EF50D880255408E2EAC0E9FFEBC0E1
:10387000EAFFEE52FC0EEFCFDBFFE26BFC0EDB50FB
:10388000E25D19E2E251EA6A400FE96E050EEA22B2
:10389000EF50E66EE251E76EFD0EDBCFE9FFFE0E64
:1038A000DBCFEAFFE750E926000EEA22E552E750B7
:1038B000EF6EE22BE3D7400EE66E400EE66E050E8D
:1038C000E66EE66A020EE66EACEC13F0256E050EAF
:1038D000E15E2550F3CFEAF0F4CFEBF00001E251C6
:1038E000E552E7CFD9FF1200D9CFE6FFE1CFD9FFEC
:1038F0000001E3510CE1FD0EDBCFE4F0FE0EDBCF67
:10390000E5F0FC0EDBCFE8F0010EE96FE36FE55266
:10391000E7CFD9FF1200D9CFE6FFE1CFD9FF030EE1
:10392000E1260001E3512DE1DF6AFD0EDBCF06F059
:10393000FE0EDBCF07F0DE5206C0DEFF07C0DDFF64
:10394000DD52DF2ADF50256E266AFF0E251802E1C0
:1039500026500BE0010EDBCFE9FFDB2A020EDBCFA6
:10396000EAFF01E3DB2AEF50ECE1FD0EDBCFE4F0F0
:10397000FE0EDBCFE5F0DF040001E86F010EE96F1A
:10398000E36F030EE15C02E2E16AE552E16EE552AB
:10399000E7CFD9FF1200D9CFE6FFE1CFD9FF030E61
:1039A000E1260001E3512EE1DF6AFD0EDBCF06F0D8
:1039B000FE0EDBCF07F0DE5206C0DEFF07C0DDFFE4
:1039C000DD52DF2ADF50256E266AFF0E251802E140
:1039D00026500CE0010EDBCFF6FFDB2A020EDBCF18
:1039E000F7FF01E3DB2A0800F550EBE1FD0EDBCF2A
:1039F000E4F0FE0EDBCFE5F0DFCFE8F00001E96B8D
:103A0000010EE36F030EE15C02E2E16AE552E16E52
:103A1000E552E7CFD9FF1200D9CFE6FFE1CFD9FFBA
:103A2000020EE1260001EC51ED1102E1000E08D07A
:103A3000ECC0E9FFEDC0EAFFEF50800B01E0010EA2
:103A4000000901E084D0030EE35D01E1E36BE35183
:103A500001E17DD0020EE35D16E1E66A000EE66E3E
:103A6000E66A010EE66E020EE66EACEC13F0256E11
:103A7000050EE15E2550F3CFECF0F4CFEDF0000140
:103A8000030EE36F64D0E30562E1400E256E266A03
:103A9000E851255C000E265803E2400EDF6E02D08E
:103AA000E8C0DFFFDF50E85DE86F000EE66F050E4F
:103AB000E76F010EDFCFDBFFE95116E1010EDB50AE
:103AC00028E0E4C0F6FFE5C0F7FF0800F550E6C0C7
:103AD000E9FFE7C0EAFFEF6EE62B000EE723E42BD9
:103AE000E523010EDB06EAD7010EDB5012E0E4C04D
:103AF000E9FFE5C0EAFFEF50E6C0E9FFE7C0EAFFF3
:103B0000EF6EE62B000EE723E42BE523010EDB0628
:103B1000EBD70001E85107E1400EDF5C02E1020E45
:103B200001D0030EE36FDFCFE6FF000EE66E050E59
:103B3000E66E010EE66E020EE66EACEC13F0256E3C
:103B4000050EE15E2550F3CFECF0F4CFEDF0020E60
:103B5000E15C02E2E16AE552E16EE552E7CFD9FFAE
:023B6000120051
:0E3B6200200E896E8B6A946893689268928A2E
:103B7000176A186A196A1950256E266AD890265055
:103B800004E6800E255C000E265809E21950EA6A08
:103B9000400FE96E040EEA22EF6A192AECD7196A7F
:103BA000400E195C09E21950EA6AC00FE96E040E72
:103BB000EA22EF6A192AF4D71200246A020E1A6E5A
:103BC000200E8914896E8B6A94689368DF0E9210B8
:103BD000926E0101E26B320E0401C05D1DE192960E
:103BE000C1C425F0266A25BE266825C0E6FF26C08A
:103BF000E6FFFA0E276E3F0E286E296A27C0E6FF01
:103C0000E66E29C0E6FFC20EE66E010EE66E1AEC05
:103C100022F02A6E070E1FD0C1C425F0266A25BEE9
:103C2000266825C0E6FF26C0E6FFEA0EE66E3F0ED8
:103C3000E66EF30E276E3F0E286E296A27C0E6FF58
:103C4000E66E29C0E6FFC20EE66E010EE66E1AECC5
:103C500022F02A6E090EE15E2A50630E245C01E117
:103C600077D02450620A71E0640A64E0030A47E0F6
:103C7000010A3AE0070A1DE0010A07E0030A03E02F
:103C8000010AEBE15ED0020E61D00401C1051A5CAD
:103C900004E1020E141401E092981A50EA6AC00F6F
:103CA000E96E040EEA22EF1C8A6E1A2A936A030E4A
:103CB0001DD08250020B16E11BC025F01CC026F05F
:103CC0001DC027F01EC028F01B06000E1C5A1D5AEE
:103CD0001E5AD8802554000E2654000E2754000E7C
:103CE0002854BBE3040E32D09490050E246EA00E2F
:103CF0001B6E860E1C6E010E1D6E1E6AAED78250A4
:103D0000040B16E11BC025F01CC026F01DC027F0D7
:103D10001EC028F01B06000E1C5A1D5A1E5AD880C1
:103D20002554000E2654000E2754000E285495E307
:103D3000060E0CD09368928894800401C1511A5CDD
:103D400002E2010E03D0630E01D0630E246E85D70C
:103D5000320E0401C05D01E19286948094689368FC
:103D6000DF0E9210926E0101E26B1200D9CFE6FFD6
:103D7000E1CFD9FFE652DF6AA00E1F6E0F0E206E54
:103D8000216A226A176A200E8914896E8B6AF90EDD
:103D9000946E9368DF0E9210926E236A800EE66E28
:103DA000E66AE66A400EE66E040EE66EE0EC20F08F
:103DB000256E050EE15E2550630E235C01E1C3D044
:103DC0001750256E266AD890265004E6800E255C92
:103DD000000E265802E3090E236E2350090A01E162
:103DE000ADD0030A01E1A8D00C0A01E184D0030A96
:103DF00052E0010A4CE0070A26E0010A10E0030A3B
:103E000005E0010AD9E19492949473D09482D00E83
:103E10001F6E070E206E216A226A020E92D082B0B7
:103E200002D0030E236E1F06000E205A215A225A7A
:103E3000D8801F54000E2054000E2154000E22542E
:103E4000BBE30A0E7ED0D00E1F6E070E206E216AD5
:103E5000226A94928050080B02E1000E01D0010EFC
:103E6000166EE8500CE0811CE66E1750172AEA6ABD
:103E7000400FE96E040EEA22E552E750EF6E8050E3
:103E8000100B01E0010E156E9484040E5AD082A02E
:103E900093D7050E56D09494155014E1060E236E58
:103EA000E80E1B6E030E1C6E1D6A1E6A14A484D7D6
:103EB0001750172AEA6A400FE96E040EEA22F1C58C
:103EC000EFFF7AD7020E0501F45D13E11704EA6AE9
:103ED000400FE96E040EEA22EF500101E75D09E1AF
:103EE000060E236EE80E1B6E030E1C6E1D6A1E6A04
:103EF00063D7010E26D080A802D0090E236E1B06C0
:103F0000000E1C5A1D5A1E5AD8801B54000E1C54F9
:103F1000000E1D54000E1E5402E3630E236E949295
:103F2000949414A649D70401320EC06F030EC16FDA
:103F30005F0EC26F42DE40D7010EDF6E9492949402
:103F4000630E236E39D7DF5003E0F368F46A07D0BD
:103F50001750256E266A17C0F3FF26C0F4FFE552FE
:103F6000E552E7CFD9FF120092928092A00E1B6E0D
:103F7000860E1C6E010E1D6E1E6A1B501C101D103D
:103F80001E1006E01B06000E1C5A1D5A1E5AF5D7BD
:103F900092828082A00E1B6E860E1C6E010E1D6E1C
:103FA0001E6A1B501C101D101E1006E01B06000E82
:103FB0001C5A1D5A1E5AF5D71200D9CFE6FFE1CF81
:103FC000D9FFFE0EDB0403E1929A809A02D0928A16
:0A3FD000808AE552E7CFD9FF120006
:063FDA000D0A5374617230
:103FE00074696E670D0A0025530044415441206CEA
:103FF000656E0025533A25642000434D44206C65CE
:104000006E3A202564200053657020303320323012
:104010003135005072656C6F6769782047504942AE
:104020002D55534220436F6E74726F6C6C65722015
:1040300076657273696F6E20362E322025530D0A15
:10404000004E6565642068656C703F204C6F6F6B37
:1040500020696E2074686520736F757263652063D4
:104060006F6465210D0A00256400656E6400766545
:104070007200747267007372710073706F6C6C0001
:10408000736176656366670072737400726561645C
:1040900000726561645F746D6F5F6D73006D6F6456
:1040A00065006C6F6E006C6F630069666300686525
:1040B0006C7000656F7400656F745F636861720097
:1040C000656F7300656F6900636C72006175746F72
:0640D0000061646472004F
:0A40D600FF0EE3CFEAFFE552FF0EF4
:1040E000E3CFE9FFE552E66AE66AD9CFE6FFDACF29
:1040F000E6FFFC0EE124D96EFF0EE220DA6EE66ADE
:10410000E66AE66A200EEF5C06E0090EEF5C03E06B
:10411000EF6603D03FD0EE50F5D72D0EEF5C03E1F4
:10412000FF0EE32A03D02B0EEF5C01E1EE502F0EC1
:10413000EF6424D03A0EEF6021D0D890F90EE33628
:10414000FA0EE336FD0EDECFE3FFFE0EDDCFE3FF1A
:10415000D890F90EE336FA0EE336D890F90EE3362E
:10416000FA0EE336FD0EE350DE26FE0EE350DD22AE
:10417000300EEE5CDE26000EDD22D9D7FF0EE3CF37
:10418000E8FFE85207E0F90EE31EE32AFA0ED8B47E
:10419000E306E31EE552E552E552FF0EE3CFDAFFF8
:1041A000E552FF0EE3CFD9FFE552E1CFE9FFE2CFC1
:1041B000EAFFED52ED52EECFF3FFEFCFF4FF120026
:1041C000FE0EE3CFE9FFFF0EE3CFEAFFE9CFF3FFF7
:1041D000EACFF4FFFB0EE35003E1FC0EE35009E0ED
:1041E000FB0EE30602E2FC0EE306FD0EE350EE6E6C
:1041F000F1D71200FF0EE3CFF8FFE552FF0EE3CF39
:10420000F7FFE552FF0EE3CFF6FFE552E66AE66AF6
:10421000E66A0900F55209E0FD0EE32A05E1FE0E0B
:10422000E32A02E1FF0EE32AF4D7FD0EE3CF05F007
:10423000FE0EE3CF06F0FF0EE3CF07F01200FD0EF7
:10424000E3CFF6FFFE0EE3CFF7FFFF0EE3CFF8FF5D
:10425000FB0EE3CFE9FFFC0EE3CFEAFFF90EE350DC
:1042600003E1FA0EE3500BE0F90EE30602E2FA0E68
:10427000E306EE500900F55C02E1F566EFD71200A7
:10428000FE0EE3CFE9FFFF0EE3CFEAFFF36AF46A25
:0C429000EE5203E0F34AF42AFBD71200C0
:04429C00120EAF6EE1
:1042A000B06AB896AC98AB8EAB88AB9A9D989D9A45
:1042B000D08E9F8AF28EAC90AB9CAC9AAC8AAC94B8
:1042C0000001E191E06B1200D9CFE6FFE1CFD9FF09
:1042D0009EB803D014D80400FBD7FE0EDB50AD6EA1
:1042E000E552E7CFD9FF12009EBA03D0040007D8E9
:1042F000FBD7AE5000D012009EBA010C000CD9CFF3
:10430000E6FFE1CFD9FFE652ABA204D0AC9AAC8A6B
:10431000AB98AB88ABA404D0AE50DF6EAC9AAC8A3D
:10432000E552E552E7CFD9FF1200D9CFE6FFE1CF42
:10433000D9FFFD0EDBCFE9FFFE0EDBCFEAFFEF502A
:1043400010E0FD0EDBCFE9FFFE0EDBCFEAFFEF5002
:10435000E66EBADFE552FD0EDB2AFE0EEAE3DB2A4B
:0A436000E8D7E552E7CFD9FF1200BD
:06436A0012010002020036
:104370000008D8040A0000010102000109024300FC
:10438000020100C0320904000001020201000524FC
:104390000010010424020205240600010524010086
:1043A000010705810308000209040100020A000058
:1043B00000070502024000000705820240000004D9
:1043C00003090434034D006900630072006F006349
:1043D00000680069007000200054006500630068F8
:1043E000006E006F006C006F0067007900200049CC
:1043F000006E0063002E003403430044004300209D
:1044000000520053002D00320033003200200045DE
:10441000006D0075006C006100740069006F006E33
:10442000002000440065006D006F007C43BF43C363
:0344300043F7430C
:0C443400D9CFE6FFDACFE6FFE1CFD9FFD9
:10444000E2CFDAFFE652E652E652E652D950F90FD1
:10445000256EFF0EDA20266E020E25C0DBFF030E4E
:1044600026C0DBFF020EDBCFE6FF030EDBCFE6FF4D
:10447000F90EDBCFE6FFFA0EDBCFE6FFFB0EDBCF5C
:10448000E6FFD950FC0FE66EFF0EDA20E66E32EC46
:1044900000F0256E070EE15C02E2E16AE552E16E92
:1044A0002550F3CFDEFFF4CFDDFFFC0EDBCFE9FFBD
:1044B000FD0EDBCFEAFFEF6ADECF25F0DDCF26F081
:1044C00025C0F3FF26C0F4FF040EE15C02E2E16ABE
:1044D000E552E16EE552E5CFDAFFE7CFD9FF1200F2
:1044E0001E0EF66E000EF76E000EF86E010109004A
:1044F000F550F46F0900F550F56F03E1F46701D052
:104500003DD00900F550EF6F0900F550F06F09003C
:10451000F550F16F09000900F550E96E0900F550FA
:10452000EA6E090009000900F550F26F0900F55024
:10453000F36F09000900F6CFF6F1F7CFF7F1F8CFE6
:10454000F8F1EFC1F6FFF0C1F7FFF1C1F8FF01018B
:10455000F25302E1F35307E00900F550EE6EF20763
:10456000F8E2F307F9D7F6C1F6FFF7C1F7FFF8C194
:0E457000F8FF0101F407000EF55BBFD7120043
:02457E00D9CF93
:10458000E6FFDACFE6FFE1CFD9FFE2CFDAFFFB0E9D
:10459000DBCF25F0FC0EDBCF26F00001800E2614C9
:1045A0001AE1FB0EDBCFE9FFFC0EDBCFEAFFEECF1B
:1045B000F3FFEDCFF4FFEE2A000EEF22F3CFE9FF79
:1045C000F4CFEAFFFD0EDBCFEFFFEF50266AF36E6C
:1045D00026C0F4FF10D0FB0EDB50FE0806E1FD0EF6
:1045E000DBCFE6FFAEEC23F005D0FD0EDBCFE6FF20
:1045F00003EC00F0E552E552E5CFDAFFE7CFD9FF53
:024600001200A6
:0E46020004500B02F3CF00F0F4CF01F00C02D5
:10461000F3500126000EF420026E04500D02F350F8
:104620000226000EF420036E04500E02F3500326FF
:1046300005500B02F3500126F4500222000E032213
:1046400005500C02F3500226F450032205500D02CF
:10465000F350032606500B02F3500226F4500322B7
:1046600006500C02F350032607500B02F3500326AA
:02467000120036
:0E46720007C013F006C012F006500D02F4CF80
:1046800005F0F3CF04F007500E02F4CF07F0F3CF9C
:1046900006F00D02F3500526F4500622E86A0722C0
:1046A00012500E02F3500526F4500622E86A072243
:1046B0000EAE5FEF23F01250065E1350075A13AE92
:0C46C000000C0D50065E0E50075A000C56
:0446CC00F36AF46A2F
:1046D000FF0EE124E96EFF0EE220EA6EED660DD0DA
:1046E000400EEF640AD05A0EEF6406D0600EEF64FD
:1046F00004D07B0EEF6001D0F32A1200F36AF46A53
:10470000FF0EE124E96EFF0EE220EA6EED6607D0AF
:104710002F0EEF6404D03A0EEF6001D0F32A12009E
:10472000000EF36E00EE00F0080E01D81200EA60F1
:1047300002D0EE6AFCD7F350E9601200EE6AFCD7B3
:1047400013EE00F023EE00F0F86A0A9C70EC22F001
:0C475000FFEC07F045EC06F0FBD7120070
:04475C00FF0EE35019
:10476000ACBA04D0AF6AAB8EAC8A949CACA2FED734
:08477000AD6EF36EF46A120055
:08477800FF0EE3502C6E1B0E36
:1047800000D001D0200EE76EE72EFED72C2EFAD7F0
:0447900000D0120043
:0C479400FF0EE350E84E1200000000D0C1
:0A47A00000D000D0E82EFAD7120076
:0647AA00303132333435DA
:0B47B0003637383961626364656600CB
:0547BB00D1405619CCAD
:1047C00040E019C840701BC440BA1BC040961CB7DB
:1047D00040FC1DB340201DAE40BC1AAA40FE1AA6E4
:1047E00040861EA240B21E9D408E1F91403A218CF1
:1047F0004074208840C821804026247A40302276A8
:1048000040242372408C236E40261B6A4000000027
:084810000000004E554C4C0065
:020000040030CA
:0100000024DB
:010001000EF0
:010002003FBE
:010003001EDE
:010005008179
:010006008178
:010008000FE8
:01000900C036
:01000A000FE6
:01000B00E014
:01000C000FE4
:01000D0040B2
:00000001FF
